:100000000C9494020C94CC020C94CC020C94CC0270
:100010000C94CC020C94CC020C94CC020C94CC0228
:100020000C94CC020C94CC020C944E0D0C94900CBD
:100030000C94041A0C94CC020C94CC020C94CC02B8
:100040000C94CC020C94CC020C94CC020C94CC02F8
:100050000C94CC020C94C6190C94CC020C94CC02D7
:100060000C94CC020C94CC020C94CC020C94CC02D8
:100070000C94CC020C94CC020C94CC020C94CC02C8
:100080000C94CC020C94CC020C94CC020C94CC02B8
:100090000C94CC020C94CC020C94CC020C94CC02A8
:1000A0000C94CC020C94CC020C94CC026D05E105AE
:1000B00075053F054305790546057C05870551050E
:1000C000D70555058B0559058F05B9055D059305C0
:1000D000C30563059905A3054A0580054D058305FC
:1000E00068059E05AF05CF05D1053B057105EA05FD
:1000F0001006160604060A061C0622062806CB066B
:10010000CB06FE06FE067807990899089908960717
:100110000A081B081B08A80ACF0A780CCF0A780C1B
:100120001B0B3E0B780C330C430CEE15F1151C1613
:100130002C1633163E16DB16DB16DB16DB16DB162B
:100140004116431648166E16911694169716BB164E
:10015000000000000000000000000000000000009F
:10016000000000000000000000000000000000008F
:10017000000000007E0F00D4FFFFFFC700000078E2
:1001800000000000000000002A2B280000000000F2
:100190000000000000000000000000290000000036
:1001A0002C1E3420212224342627252E362D3738A4
:1001B000271E1F202122232425263333362E3738AD
:1001C0001F0405060708090A0B0C0D0E0F1011126B
:1001D000131415161718191A1B1C1D2F3130232D37
:1001E000350405060708090A0B0C0D0E0F10111235
:1001F000131415161718191A1B1C1D2F3130354CE6
:1002000005010980A101850319012AB700150126FE
:10021000B700950175108100C0050C0901A1018589
:100220000419012AA002150126A00295017510816A
:1002300000C005010906A1018506050719E029E7A7
:10024000150025019508750181020507190029EFA0
:100250001500250195F07501810205081901290590
:10026000950575019102950175039101C00660FF26
:100270000961A1010962150026FF0095207508811A
:10028000020963150026FF00952075089102C0053C
:10029000010906A101050719E029E71500250195C7
:1002A000087501810295017508810105071900296A
:1002B000FF150026FF009506750881000508190145
:1002C0002905950575019102950175039101C009F4
:1002D000025B00030100A0FA090400000103010110
:1002E00000092111010001224000070581030800D7
:1002F00001090401000203000000092111010001AD
:1003000022220007058203200001070503032000C5
:10031000010904020001030000000921110100018C
:10032000226D000705840320000112010002000075
:100330000008686168700001010200012603700076
:10034000690061006E006F0066006F00720074004B
:100350006500200068006F00740073007700610082
:10036000700000000E0341006C006900630065002E
:10037000480000000403090429003B003D003F0041
:10038000410043004500460048003A003C003E0062
:1003900040004200440068004700000035001F0094
:1003A00021002300250027002E0049004B001E00DD
:1003B00020002200240026002D002A004A00000010
:1003C0002B001A0015001C000C00130030004C001C
:1003D0004E00140008001700180012002F00310012
:1003E0004D0000003900160009000B000E0033001C
:1003F000280000000000040007000A000D000F00A4
:100400003400000000000000E1001B001900110092
:10041000360038000000520000001D0006000500F4
:10042000100037000000E50000000000E000E200DE
:1004300000000000E6000000215250004F00E300E1
:1004400000002C0000000000E700E4005100000064
:100450000100010001000100010001000100010094
:100460000100010001000100010001000100010084
:100470000100000001000100010001000100010075
:100480000100010001000100010001000100010064
:100490000100010001000000010001000100010055
:1004A0000100010001000100010001000100010044
:1004B0000100010001000100010000000100010035
:1004C0000100010001000100010000000000010026
:1004D0000100010001000100010000000000000017
:1004E0000100010001000100010001000000010005
:1004F00000000100010001000100010000000100F6
:1005000000000000010001000000000001000000E8
:1005100001000100010001000000010000000000D6
:10052000010001000100000011241FBECFEFDAE03E
:10053000DEBFCDBF04B603FE18C080919B02909130
:100540009C02A0919D02B0919E028730904BA740E3
:10055000B04B59F410929B0210929C0210929D0293
:1005600010929E02E0E0F8E3099511E0A0E0B1E00E
:10057000E4EAF9E302C005900D92A236B107D9F77B
:1005800022E0A2E6B1E001C01D92AB39B207E1F76B
:100590000E94AD130C94D01C0C9400000E94FE1716
:1005A0002FE78AE196E0215080409040E1F700C0BB
:1005B00000009CE088E10FB6F894A8958093600055
:1005C0000FBE90936000FFCFA7E1B0E0EAEEF2E04B
:1005D0000C949B1C4B8B5C8B6D8B7E8B8F8B61117A
:1005E0001092100286E09E01235F3F4FD901E82F51
:1005F0001D92EA95E9F795E0FE017396D901019005
:100600000D929A95E1F79C894E895F897B897D8758
:100610009E876F87598B488BF901DE0117960190F1
:100620000D928A95E1F7CE0107960E94261281115C
:100630003EC086E0FE013796DE01119601900D92D4
:100640008A95E1F7FF81E8856A857B8561157105EB
:1006500031F0EF3F31F481E0FF3F19F403C081E056
:1006600001C080E080FD23C02091BD0130E0C901C0
:100670000196877099274091EE0150E08417950705
:1006800079F1F983EA837D836C8396E0929FD001B0
:10069000939FB00D1124A254BE4FFE0131960190DC
:1006A0000D929A95E1F78093BD010E94B31116E077
:1006B0008091EE019091BD018917F9F0189FC0015A
:1006C000112482549E4F0E9426128823B1F08091FB
:1006D000EE0190E00196877099278093EE01E8CFB4
:1006E0000E94FE171092BD011092EE01E7EBF1E0BF
:1006F00086E0DF011D928A95E9F76796E3E00C94A6
:10070000B71CADE0B0E0E7E8F3E00C948C1CFC0112
:100710008081918123813481232B31F09F3F31F4FB
:1007200091E08F3F19F403C091E001C090E090FD8B
:100730003EC57F0185E0DE01199601900D928A95F4
:10074000E1F7F701228189859A85222349F00E94E9
:100750000317182F682F89859A850E94731703C085
:100760000E943F17182F69857A85812F0E94710F8B
:100770008C01F7018281882309F42CC19801225051
:1007800037472031310508F041C18FEF93E00E94D7
:100790003D1C811129C1025036EDA32EBB24B39418
:1007A000002379F0A114F4E0BF0609F41DC1C501CE
:1007B0000E943D1C811101C001502FEFA21AB20A04
:1007C000EFCFCE0101962C0188E0F20111928A95BB
:1007D000E9F72AE0322E85010F5F1F4FC5010E9405
:1007E0003D1C89831A82882309F4FEC0813009F0F8
:1007F00041C06501F2E0CF0ED11CC8010E943D1C32
:100800008A83882309F4F0C09FEF980F933060F437
:1008100023E0A20EB11CC6010E943D1C8B838823DD
:1008200009F4E2C01C8229C0843031F54E0133E066
:10083000830E911C02E010E056018FEFA81AB80A4F
:10084000C6010E943D1CF40181934F01882309F4E5
:10085000CBC08C3741F4E2E0F0E0EC0FFD1FE00F7D
:10086000F11F10820AC00F5F1F4F6501073011058D
:1008700019F7BAC0580101C056018201F801208160
:10088000222309F4A8CF213009F04CC081818130A6
:1008900049F46801F2E0CF0ED11CF80182810E9478
:1008A00042190AC0823051F46801F2E0CF0ED11C27
:1008B000F80182810E948818860189C0833049F43A
:1008C0006801F2E0CF0ED11CF80182810E942F183E
:1008D000F3CF843019F00F5F1F4F79C0F8012281E8
:1008E0000E5F1F4F80E090E030E0205331092A3046
:1008F000310568F4389EA001399E500D1124C901BC
:10090000840F951F0F5F1F4FF8012081EDCF0097D7
:1009100009F45DC0EFECF7E03197F1F700C000009B
:100920000197F5CFE22FF0E0E058FE4F2490822FA0
:1009300086958695869590E0FC01E059FE4F64907F
:100940002770712C022E02C0759467940A94E2F706
:10095000F1E06F227724FC01E05AFE4F8490912C45
:10096000022E02C0959487940A94E2F731E0832224
:100970009924FC01E05BFE4FC490D12C02C0D594B9
:10098000C7942A95E2F781E0C822DD24611471043E
:1009900019F081EE0E9488188114910419F086EEF6
:1009A0000E948818822D0E9442198114910419F026
:1009B00086EE0E942F186114710419F081EE0E94D6
:1009C0002F18C114D10419F08CE20E9442190F5F54
:1009D0001F4F54CF011537E7130709F042C181E0DB
:1009E0000E94AB170E94B9098091EF01877009F44A
:1009F000DEC3F7018281882309F4D9C3809166019F
:100A000082FFD5C382E00E947F11D1C30115F7E7B1
:100A10001F0711F481E005C0013027E7120721F418
:100A200082E00E94B817DECFF801E851FC47E730BA
:100A3000F10508F4E5C0882309F45BC110928F0228
:100A4000C8019057839708F013C184E090E00E949A
:100A5000451C9093660180936501F801E150F047D1
:100A6000E232F10520F4EA5AFF4F0C947F1C80918A
:100A700065018160ACC0809166018860B4C08091DE
:100A800065018260A4C08091650120C080916501EC
:100A900088609DC0809166011EC080916601826061
:100AA000A2C080916501806192C0809165018062E1
:100AB0008EC08091650180648AC00E94FE1780917B
:100AC0006501806884C080916501886084607FC012
:100AD000809166018260816086C0809165018E7F11
:100AE00076C080916601877F7EC0809165018D7F91
:100AF0006EC08091650120C080916501877F67C0CD
:100B0000809166011EC0809166018D7F6CC08091CE
:100B100065018F7E5CC0809165018F7D58C080919A
:100B200065018F7B54C00E94FE17809165018F770D
:100B30004EC080916501877F8B7F49C0809166019F
:100B40008D7F8E7F50C08091650182FB222720F926
:100B500091E0922790FB82F990FB83F938C0809155
:100B60006601982F909591708E7F892B90FB81F96B
:100B70003AC08091650186FB222720F991E09227F7
:100B800090FB86F924C00E94FE178091650187FBC7
:100B9000222720F991E0922790FB87F918C061E0A5
:100BA00001C060E08EE090E00E944B1C1EC080916E
:100BB000650184FB222720F991E0922790FB84F9BC
:100BC00006C080916501982F909590FB80F98093E5
:100BD00065010BC08091660183FB222720F991E01B
:100BE000922790FB83F98093660160916501709173
:100BF000660184E090E00E94691C0E94FE17F4CE1A
:100C0000E858FF4F0C947F1C06E221EE41EE6AE1AA
:100C10007CE723C007E225EE45EE6BE17CE71DC0D3
:100C200006E221EE40EE68E17CE717C007E225EE20
:100C300044EE69E17CE711C006E221EE42EE6CE190
:100C40007CE70BC007E225EE46EE6DE17CE705C0D0
:100C500008E221E045EE6EE17CE7C7010E94E11A5F
:100C6000C3CE013097E7190709F0DECE82E0B8CE97
:100C70000631ECE71E0709F47AC203309CE7190736
:100C800021F140F40115FCE71F0789F001301C47F2
:100C900011F134C00B353CE7130739F10C358CE703
:100CA0001807D9F00A351C4749F581E01FC00E949A
:100CB000FE17EFE7FAE126E0E150F0402040E1F7CF
:100CC00000C000000E94A2198FCE6FEF7FEF80E07E
:100CD00090E00E94691C0E94CE028091660182FB16
:100CE000882780F991E0892701C080E00E949C114B
:100CF00005C00631FCE71F0709F449C2F7018281EC
:100D000000811181882349F0C8010E940317D82E61
:100D1000682FC8010E94731704C0C8010E943F17C2
:100D2000D82EB8018D2D0E94710F0E947F0FB82E12
:100D3000192F982EF7010281A580A2949FE0A92285
:100D40008091EF018770B9F00023A9F0812F807F97
:100D5000803421F080E28B0D883068F0809166014C
:100D600082FF09C082E00E947F118091EF018770AD
:100D7000DD24D3948111D12CC12EC2948FE0C822DE
:100D80008C2D90E08C30910508F0D3C1FC01E15826
:100D9000FF4F0C947F1C812F807F1F70882311F0E0
:100DA0001295107F0023B9F0112309F4B0C180E23D
:100DB0008B0D883010F0911006C090911102192B04
:100DC0001093110205C090911002192B109310027C
:100DD0000E942A119CC18B2D0E942F18112309F407
:100DE000A8C180E28B0D883088F1992079F11095A7
:100DF000909110021923109310022BC0812F807F35
:100E00001F70803211F01295107F8B2D992029F0E0
:100E1000F1E09F1609F441C04FC08091660182FD48
:100E20001BC0002369F0112339F090911102192B96
:100E3000109311020E942A1180E00E94881879C143
:100E400080E00E942F18112309F473C1812F0E94A2
:100E500023110E942A116DC1002381F0809112029A
:100E6000AA2051F021E0A21207C0182B181709F48C
:100E700060C1109312025DC1812B16C0A11003C086
:100E80000E941D1131C031E0A31609F452C1812F17
:100E90000E941E180E941D114CC1002341F085E0E4
:100EA0008A1508F446C1812F0E94251842C194E09A
:100EB0009A1508F43EC118C0002349F0AA2099F3FE
:100EC000F701858180FF23C18F708583ECCFAA2035
:100ED00059F0893309F02AC1FFEF23EF31E0F150D7
:100EE00020403040E1F720C1812F0E941E1821C10F
:100EF000812F86958695837019F0813061F019C134
:100F0000002321F08B2D912F937002C080E090E0A0
:100F10000E94AF1A14C1002321F08B2D912F9370E2
:100F200002C080E090E00E948A1A09C1812F83707C
:100F3000A9F5011102C14B2D429546954770440F0A
:100F4000440F8B2D8F7090E09C01042E01C0220F66
:100F50000A94EAF7B4FE08C08FE090E001C0880F61
:100F60004A95EAF7809501C080E0169516951370B2
:100F7000123069F088F490912E02113019F0822B12
:100F8000892302C0922B892B0E94C417D6C0822BC2
:100F900090912E028927F8CF822BF6CF002319F0EB
:100FA000812F817001C08695882309F4C6C04B2D1E
:100FB000429546954770440F440F8B2D8F7090E0FB
:100FC0009C01042E01C0220F0A94EAF7B4FE08C067
:100FD0008FE090E001C0880F4A95EAF7809501C044
:100FE00080E0169516951370123059F078F49091B0
:100FF0009601113019F0822B892309C0922B892B7D
:1010000006C0822B90919601892701C0822B0E94F5
:10101000A81793C01F70002339F0812F0E94B817C2
:101020008B2D0E94251889C08B2D0E941E18812FA0
:101030000E94AB1782C08B2D92EF991681F1991502
:1010400038F0E0EF9E1659F0F1EF9F1619F15BC0F2
:1010500023EF921659F134EF9316C1F054C00023D8
:1010600081F084E08A1508F464C01F7181E090E08B
:10107000012E01C0880F0A94EAF790919601892702
:1010800020C095E09A1508F454C0EFCF8091660116
:1010900082FD1AC0002329F0812F8F7127C0002301
:1010A000D9F3812F8F710E94AB1743C0002341F009
:1010B0001F7181E0012E01C0880F0A94EAF701C078
:1010C00080E00E94A81735C0002399F01F71812F7E
:1010D0000E94B8178091660182FF07C0E8E01E9F5A
:1010E000C001112483608093EF01812F0E94B81703
:1010F00020C081E00E947F11F1E0FA15D0F482E077
:101100000E947F1116C0002321F0AA2029F28B2D06
:1011100094CEAA2031F2893349F42FEF33EF81E0E6
:10112000215030408040E1F700C000008B2D0E942C
:101130002F1888EF8C0D843010F40E94D41ADD2013
:10114000B1F18091EF0180FD32C0F70112828595E7
:10115000859585950E94B817C7010E9481038091EB
:10116000EF018595859585950E94AB1720C08091EC
:1011700011028A7A91E009F490E090936401811160
:1011800012C069E287E991E00E94551A09C0809176
:10119000640181110AC069E287E991E00E942D1A79
:1011A0000E942A1121CC65E3EDCF65E3F5CF2D96A2
:1011B000E2E10C94A81C80918E0187FF11C0809100
:1011C000E80082FD05C080918C018111F8CF11C02B
:1011D0008091E8008B770BC080918C01882349F0C7
:1011E0008091E80080FFF8CF8091E8008E778093AF
:1011F000E8000895982F973068F59093E9009817C4
:1012000039F07091EC002091ED005091F00003C096
:10121000242F762F50E021FD02C09F5FECCF30914C
:10122000EB003E7F3093EB003091ED003D7F30933B
:10123000ED003091EB0031603093EB007093EC00E7
:101240002093ED005093F0002091EE0027FDE5CFB4
:1012500080E008958F708093E90081E008952091E7
:101260009401309195012617370748F061157105F3
:1012700039F42091E8002E772093E80001C0B901ED
:10128000FC0120E06115710579F180918C018823C2
:10129000F1F18530F1F18091E80083FD3CC080914F
:1012A000E80082FD2EC08091E80080FFEBCF209106
:1012B000F3008091F20090E0922B6115710551F0DE
:1012C0008830910538F421912093F1006150710923
:1012D0000196F3CF21E0089709F020E08091E80023
:1012E0008E778093E800CECF2111CFCF0AC08091B6
:1012F0008C01882361F0853061F08091E80083FDE6
:101300000AC08091E80082FFF2CF80E0089582E079
:10131000089583E0089581E00895089543E050E042
:10132000BC0184E00E9464190895CF93DF93EC011F
:1013300080910001811105C048E050E0BE0181E0CC
:101340000BC08091650187FF03C040E284E002C0CA
:1013500048E081E050E0BE010E94641980E2FE0195
:10136000AAE6B1E001900D928A95E1F7DF91CF9165
:10137000089580919601982F9670963011F48860A8
:1013800001C0877F0E94A8170895AAE2B0E0EBECA5
:10139000F9E00C949B1CEEE8F1E086E991E02091E5
:1013A000F10021938E179F07D1F780918F01833031
:1013B00009F463C030F4813071F0823009F49DC0CB
:1013C000B4C08A3009F489C08B3009F46EC089300A
:1013D00009F0ABC020C080918E01813A09F0A5C010
:1013E0008091E800877F8093E8008091920190913E
:1013F0009301892B21F460E28AE691E003C060E06A
:1014000080E090E070E00E942F098091E8008B77E7
:101410008093E8008AC080918E01813209F085C0F6
:101420008091920190919301009719F0029709F031
:101430007CC08091E800877F8093E8008091E8007D
:1014400082FD05C080918C018111F8CF6EC0209182
:10145000F3008091F20090E0922B029731F480919A
:10146000F100813011F0863021F48091F1008093F9
:1014700069018091E8008B7754C080918E01813A98
:1014800009F053C08091920190919301892B09F04A
:101490004CC08091E800877F8093E8008091E8004D
:1014A00080FFFCCF8091000137C080918E01813296
:1014B000E1F58091920190919301892BB1F5809192
:1014C000E800877F8093E8000E94DB08809190010C
:1014D000809300010E94FE1728C080918E01813206
:1014E00021F58091E800877F8093E8000E94DB0867
:1014F000809191018093680118C080918E01813A9A
:10150000A1F48091E800877F8093E8008091E80053
:1015100080FFFCCF809168018093F1008091E8000A
:101520008E778093E8000E94DB088091E80083FFBB
:10153000DFC180918E0190918F01492F50E04A3098
:10154000510508F0D5C1FA01E557FF4F0C947F1CF7
:10155000803821F0823809F0CBC108C080918A011F
:1015600090918B01992389F082600FC08091920144
:101570008F70873008F0BCC18093E9008091EB0048
:1015800085FB882780F91092E9009091E800977F09
:101590009093E8008093F1001092F10070C1282F21
:1015A0002D7F09F0A5C1882319F0823061F0A0C118
:1015B00080919001813009F09BC1933009F080E067
:1015C00080938B012EC08091900181112AC080915F
:1015D00092018F702FEF280F263008F089C1809379
:1015E000E9002091EB0020FF1CC0933021F4809192
:1015F000EB00806214C09091EB0090619093EB003F
:1016000021E030E0A90102C0440F551F8A95E2F79E
:101610004093EA001092EA008091EB00886080938A
:10162000EB001092E9008091E800877F8093E8004A
:101630000E94DB085DC181115BC1109190011F7791
:101640008091E3008078812B8093E3008091E80013
:10165000877F8093E8000E94DB088091E80080FF8C
:10166000FCCF8091E30080688093E300111102C0F9
:1016700082E001C083E080938C013AC180588230BF
:1016800008F036C120919001309191012C3D53E03A
:10169000350779F583E08A838AE289834FB7F89426
:1016A000DE01139620E03EE051E2E32FF0E050939C
:1016B0005700E49120FF03C0E295EF703F5FEF70A9
:1016C0008E2F90E0EA3010F0C79601C0C0968D933F
:1016D0009D932F5F243149F74FBF8091E800877FAA
:1016E0008093E8006AE270E0CE0101960E942F0923
:1016F000B4C08091920190919301432F55274330BC
:101700005105A9F068F44130510509F400C1423097
:10171000510509F0EDC08BE590E0EFECF2E04BC035
:101720004132510529F14232510589F1E1C0C90127
:10173000992781309105A1F058F0029709F0D8C09F
:10174000ECE3F3E0E4918E2F90E0ECE3F3E030C0C3
:10175000E4E7F3E0E4918E2F90E0E4E7F3E028C0C3
:10176000E4E6F3E0E4918E2F90E0E4E6F3E020C0BD
:101770008330910508F0BCC0880F991FFC01EE5E14
:10178000FE4F0190F081E02D89E090E014C083309D
:10179000910508F0ADC0FC01EE0FFF1FE45FFE4FA6
:1017A0000190F081E02DDC01A75FBE4F8C9190E0AD
:1017B000009709F49DC02091E800277F2093E8005E
:1017C00020919401309195012817390708F4C90137
:1017D00040E0009789F120918C01222309F43DC05B
:1017E0002530D9F12091E80023FD37C02091E80091
:1017F00022FD2FC02091E80020FFEBCF4091F300A5
:101800002091F20030E0342B009759F02830310558
:1018100040F444914093F100319601972F5F3F4F80
:10182000F3CF41E02830310509F040E02091E80095
:101830002E772093E800CDCF4111CDCF0AC0809103
:101840008C01882351F0853041F08091E80083FDC0
:1018500004C08091E80082FFF2CF8091E8008B778E
:101860008093E80045C0803809F042C08091E800CC
:10187000877F8093E80080918D018093F1008091B3
:10188000E8008E77D3CE811133C080919001909182
:1018900091019927029764F58091E800877F8093F2
:1018A000E8001091900110938D010E94DB08111146
:1018B00006C08091E30087FD02C081E001C084E0A2
:1018C00080938C0142E061EC81E00E94FA0842E2E0
:1018D00061EC84E00E94FA0842E261EC82E00E943E
:1018E000FA0842E260EC83E00E94FA0880918C01E1
:1018F0008091E80083FF10C08091E800877F80938B
:10190000E8008091EB0080628093EB0005C082E1EB
:1019100090E0EAE2F3E04FCFAA96E3E00C94B71C24
:101920001F920F920FB60F9211242F933F934F9354
:101930005F936F937F938F939F93AF93BF93CF9357
:10194000DF93EF93FF93C091E900CF708091EC009B
:10195000D82FD17080FDD0E81092E9008091F0007E
:10196000877F8093F00078940E94C5091092E90067
:101970008091F00088608093F000CD2BCF70C093F1
:10198000E900FF91EF91DF91CF91BF91AF919F91CE
:101990008F917F916F915F914F913F912F910F9018
:1019A0000FBE0F901F901895E8EDF0E080818E7FBC
:1019B00080831092E2001092DA001092E100A0EE13
:1019C000B0E08C9181608C9380818F77808319BC8B
:1019D000A7EDB0E08C918E7F8C9380818F7E808389
:1019E000109267010895A0E0B0E0E9EFFCE00C94EC
:1019F000961CC8EDD0E088818F7E8883E7EDF0E00B
:101A000080818160808384E082BF81E08093670170
:101A100088818E7F888302EE10E0F8011082109298
:101A2000DA0081EEC82ED12CF601108288818F77E2
:101A3000888388818068888388818F7D888319BCAA
:101A400010928C0110928D0110928B0110928A01DC
:101A500090EEE92EF12CF70180818B7F80838881C5
:101A60008160888342E060E080E00E94FA08F6012D
:101A700080818E7F8083F801808181608083808176
:101A800088608083F70180818E7F80838881806178
:101A90008883CDB7DEB7E8E00C94B21C1F920F929A
:101AA0000FB60F9211242F933F934F935F936F9331
:101AB0007F938F939F93AF93BF93EF93FF93809107
:101AC000E10082FF09C08091E20082FF05C08091A1
:101AD000E1008B7F8093E1008091DA0080FF28C0D5
:101AE0008091D80080FF24C08091DA008E7F80939F
:101AF000DA008091D90019BC80FF16C082E089BD50
:101B000009B400FEFDCF81E080938C0180916701D4
:101B100081110EC00E94D40C0E94F30C8091E2004F
:101B200084608093E20004C010928C0110926701DF
:101B30008091E10080FF17C08091E20080FF13C018
:101B40008091E2008E7F8093E2008091E2008061CC
:101B50008093E2008091D80080628093D80019BC05
:101B600085E080938C018091E10084FF2FC08091FB
:101B7000E20084FF2BC019BC82E089BD09B400FEDD
:101B8000FDCF8091D8008F7D8093D8008091E100B7
:101B90008F7E8093E1008091E2008F7E8093E2004F
:101BA0008091E20081608093E20080918D01882322
:101BB00011F084E007C08091E30087FD02C081E05E
:101BC00001C083E080938C0180918C018091E100C1
:101BD00083FF27C08091E20083FF23C08091E10052
:101BE000877F8093E10082E080938C0110928D01C9
:101BF0008091E1008E7F8093E1008091E2008E7FF2
:101C00008093E2008091E20080618093E20042E0F4
:101C100060E080E00E94FA088091F0008860809384
:101C2000F000FF91EF91BF91AF919F918F917F91C4
:101C30006F915F914F913F912F910F900FBE0F9039
:101C40001F9018952091E4003091E50095E64091B1
:101C5000EC00842F817040FF23C08091E80080FD5C
:101C60001DC080918C01882399F0853099F0809176
:101C7000EB0085FD11C04091E4005091E500241770
:101C8000350729F3915011F09A01E1CF84E00895CE
:101C900082E0089583E0089581E0089580E008954A
:101CA0004091E80042FFDDCF089580E008959091D3
:101CB000650192FF0DC0282F2871283019F4877F05
:101CC000846006C0282F2471243011F48B7F886033
:101CD00093FF0DC0282F2871283119F4877E846165
:101CE00006C0282F2471243111F48B7E8861209145
:101CF000660120FF0DC0382F3871383019F4877F06
:101D0000816006C0382F3171313011F48E7F8860C8
:101D100021FF0DC0282F2871283119F4877E816199
:101D200006C0282F2171213111F48E7E886194FD27
:101D3000877E0895F894E82FE295EF70F0E031A1E6
:101D4000282F2F7081E090E001C0880F2A95EAF7D4
:101D5000982F9095932391A392A1892B82A3789495
:101D60000895A8E1B0E0E7EBFEE00C948E1CAE0114
:101D70004F5F5F4F7A0188E1FA0111928A95E9F786
:101D80000DE411E06A0199E5492E91E0592E66248F
:101D90006394712C32E6832E31E0932EF80180811A
:101DA0008F3F09F446C0F894E82FE295EF70F0E019
:101DB00021A18F70A30102C0440F551F8A95E2F73D
:101DC000CA01922F982B91A392A18095892382A377
:101DD000789400C0E9E5F1E021E030E0A12CB12CDD
:101DE00041914F3F89F0A42FA295AF70B0E090963B
:101DF0008C9190E04F7002C0959587954A95E2F7D7
:101E000080FD02C0C90102C080E090E0A82AB92A82
:101E1000220F331F8E169F0619F7F80180818F3F1E
:101E200011F00E949A0EF0E5FA95F1F7F601B182F1
:101E3000A0820F5F1F4FF2E0CF0ED11C401651065B
:101E400009F0ACCF48E150E0B70186E192E00E9492
:101E5000C31C892B89F088E1F701A6E1B2E001906B
:101E60000D928A95E1F781E0809315020E94F8199E
:101E7000909314028093130280911502811102C085
:101E800080E02BC020911302309114024FB7F894D8
:101E90008091970290919802A0919902B0919A0234
:101EA0004FBF821B930B059758F348E150E066E162
:101EB00072E08BE492E00E94C31C892B59F088E108
:101EC000E6E1F2E0ABE4B2E001900D928A95E1F731
:101ED00081E001C080E0109215026896E0E10C9468
:101EE000AA1C7C3048F4693038F4823028F4462F3C
:101EF000672F0E94C21B089580E090E00895CF9361
:101F0000DF938238910569F1B0F48133910509F4CA
:101F100077C048F48932910509F469C08A32910585
:101F200009F473C092C08533910509F45BC089330D
:101F30009105B9F08AC0833E910591F138F4803E55
:101F40009105D1F0823E910531F17FC0863E910529
:101F5000D9F1873E9105E9F1843E910509F075C0FC
:101F600028C02091650120FD5BC021FD59C0209152
:101F7000660123FD61C069C08091650180FD4AC092
:101F80008091660180FF4CC08091650184FD50C145
:101F900083EE90E04FC18091650182FF3EC0F4CF97
:101FA0008091650182FD39C08091660180FD38C055
:101FB000EBCF8091660181FF39C08091650184FD7E
:101FC00037C187EE90E036C18091650183FF2BC059
:101FD000F4CF8091650183FD26C08091660181FD6B
:101FE00025C0EBCF8091650185FD26C022C0809180
:101FF000650185FD1EC08091660183FF1DC00AC07A
:102000008091650186FD1BC01DC08091650186FD24
:1020100019C015C089E390E00DC182EE90E00AC1BD
:1020200080EE90E007C186EE90E004C184EE90E07F
:1020300001C185E390E0FEC089E290E0FBC08AE246
:1020400090E0F8C081E390E0F5C0EC01811530E547
:10205000930708F053C0811560E4960720F0CE0185
:102060009F70906AE7C0803E910588F58D3C910590
:1020700018F0CE019065DEC0883A9105C0F4853A2B
:10208000910550F08C2F855AC82FD0E0C85EDE4FE6
:10209000888190E09064CEC08130910509F4C5C07C
:1020A00008F4C6C0049708F4C3C0CE01C3C0813C85
:1020B000910508F0BDC08C2F885AC82FD0E0CC0FF6
:1020C000DD1FC55EDE4F888199819464B3C08115A0
:1020D000904258F08D2F8F710E94570E282F2F712C
:1020E000CE0199279062922BA5C0C11581E0D80737
:1020F000E0F6C83ED10508F09BC0D7CFC03692E5C8
:10210000D90708F053C0C03422E5D207B8F08C2FAD
:102110008F718695869570E2879FA00111248C2F80
:10212000837021E030E0B90102C0660F771F8A9505
:10213000E2F7CB019C68842B952B7CC0C03232E542
:10214000D30740F08C2F8F7190E0982F8827816FF4
:10215000906A70C0C11562E5D607B0F08C2F8695E5
:10216000869520E2829FA00111248C2F837021E0AC
:1021700030E0B90102C0660F771F8A95E2F7CB0104
:10218000842B952B9D6856C08C2F8F710E94570E03
:1021900095E0D695C7959A95E1F7CF70D0E0DC2F02
:1021A000CC27D0699E01282BC90144C0C03A72E5F2
:1021B000D70708F58C2F8F71C03892E5D907A8F49E
:1021C0008695869570E2879F900111248C2F8370ED
:1021D00041E050E0BA0102C0660F771F8A95E2F72E
:1021E000CB019A68822B932B25C090E0982F8827EB
:1021F000846F906A1FC0C03C22E5D20750F48C2F38
:102200008F710E94570E8F7190E0982F88279062EF
:1022100011C0C03E32E5D30758F4CE018F71992723
:10222000982F8827806F906A05C081E090E002C0F7
:1022300080E090E0DF91CF910895809112028111AA
:102240001092120208958095909111028923809333
:10225000110208959091110280911002982B909391
:102260009701809112028823D9F0892B80939701DE
:1022700080910001882331F08091650187FF02C0C1
:102280008EE101C086E0E9E9F1E090E0815028F0BC
:1022900021912223D9F39F5FF9CF91110E941D1143
:1022A00040E250E060EF71E087E991E00E94C31CDA
:1022B000892B21F180E2E7E9F1E0A0EFB1E00190A4
:1022C0000D928A95E1F7E0919202F0919302309796
:1022D000A9F080910001882359F08091650187FF62
:1022E00007C0809197018093980186E080939701C1
:1022F0000280F381E02D87E991E00995089520910E
:10230000EF01809582238093EF01982F977099F4C5
:1023100030E0482F082E000C550B2417350759F0D4
:102320009091660192FF07C08595859585950E94DD
:10233000AB171092EF0108959091660192FB22274E
:1023400020F9281779F080FB92F99093660160914B
:1023500065017091660184E090E00E94691C82E052
:102360000E947F1108958091EE019091BD0189171F
:1023700019F08F5F8770FBCF08950F931F93CF9352
:10238000DF938091BC0182958F7009F05AC08091D3
:10239000B901882309F455C08091EE011091BD0167
:1023A0006091B7017091B801C091BA01D091BB01A1
:1023B00091E06F3F09F090E0292F06E0811709F4C2
:1023C00040C0209721F07F3F21F030E003C031E092
:1023D00001C0322F90E030FD31C0089FF001099F0D
:1023E000F00D1124DF01A254BE4F11963C911197BC
:1023F000371324C03C91361321C012963C9112979A
:1024000031111CC013964D915C9114974C1B5D0BC0
:10241000483C510598F48091BC018F708061809395
:10242000BC01ED53FE4F80818F708061808387EB0C
:1024300091E00E9481030E94B31103C0019687704E
:10244000BDCFDF91CF911F910F910895A1E1B0E031
:10245000ECE2F2E10C94931C8C0185E0F801DE01C2
:102460001D9601900D928A95E1F7F801E280909116
:10247000B7016091B8014091BA015091BB0141157B
:10248000510531F06F3F31F481E09F3F19F403C0F3
:1024900081E001C080E0F82FF1709F2E80FD1BC10C
:1024A000F80130812181C380D48087EBA82E81E0A0
:1024B000B82EF090B901F601E41BF50BFF2009F4EA
:1024C000C7C08091BC01E83CF10508F092C0482FDC
:1024D000407F09F051C0621311C093130FC0FE2C4E
:1024E000E1100CC08F7080618093BC01C5010E9417
:1024F00081038091BC01F80185832AC1C114D104F4
:1025000031F02F3F31F481E03F3F19F403C081E007
:1025100001C080E080FD03C081E08E2502C080E024
:1025200090E0F82FF170FF2E80FF1CC08091EE012B
:102530004091BD0156E0841709F4E8C090E0589F2F
:10254000F001599FF00D1124E254FE4F61812613D2
:1025500006C06081631303C06281E61203C0019666
:102560008770E9CFFE2CEE2009F4F2C08091BC0107
:1025700081608093BC0149C0621306C0931304C0FC
:10258000E11002C0F80186C0C8010E94C717882365
:1025900051F1EE2041F12091BC01822F82958F7084
:1025A00090E0029774F08091B7019091B8019887FC
:1025B0008F831986DB86CA862C87CE0107960E94F8
:1025C000810386E0F801A7EBB1E001900D928A95B6
:1025D000E1F70E94BD110AC06217C9F0C8010E944C
:1025E000C71781111EC0C8010E948103FF24F39404
:1025F000AFC0482F407F81F787EB91E00E948103B5
:1026000086E0F50111928A95E9F7F12CA1C09313A8
:10261000E5CFE110E3CFF8018583C8010E94810373
:1026200054C0EE2001F32091BC01822F82958F705F
:1026300090E0029734F28091B7019091B8019A83AB
:1026400089831B82DD82CC822E83CE010196B7CF97
:10265000E83CF105D0F5FE2CEE2029F2621327C0EC
:10266000931325C02091BC0120FD18C0822F8295B4
:102670008F70482F50E04115510581F0F8012583F6
:102680004F30510541F08F5F982F9295907F822FA8
:102690008F70892B8583C8010E94810386E0F80131
:1026A000A7EBB1E001900D928A95E1F751C0C80106
:1026B0000E94C717811185CF8091BC0181608093F2
:1026C000BC01C8010E94810343C086E0F50111925C
:1026D0008A95E9F73DC0EE2009F485CFC8010E9434
:1026E000C717F82E882309F47ECF86E0F801A7EB00
:1026F000B1E001900D928A95E1F78091B701909138
:10270000B8010E9432170E94BD1122C03D872E875A
:102710008D859E850E943217292F22952F70223099
:1027200028F49F7039F0811105C00BC0243028F4C3
:102730009F7049F4805E883020F0C8010E948103B8
:102740009F2CF92C05C0F8019581907F99F7F9CF5E
:102750008F2D6196EBE00C94AF1CACE2B0E0E3EBA4
:10276000F3E10C948C1C85B7806885BF85B78068C1
:1027700085BF84B7877F84BF0FB6F894A8958091F2
:102780006000886180936000109260000FBE90E04E
:1027900080E80FB6F89480936100909361000FBEBB
:1027A00085E59EE090936301809362010E94D40CC2
:1027B0000E94F30C8091E20084608093E2007894A0
:1027C00080918C018823A1F01091E9001F709091F5
:1027D000EC00892F817090FD80E8182B1092E900A1
:1027E0008091E80083FD0E94C5091F701093E900E5
:1027F00082E084BD93E095BD9DE797BD80936E0018
:102800000E94241C811102C00E94141C0DE411E0DE
:10281000D8018D918D018F3F11F00E949A0EB1E089
:1028200009351B07A9F709E511E0F80181918F012E
:102830008F3F11F00E949A0EF1E002361F07A9F7B0
:1028400088E1EBE4F2E0DF01282F1D922A95E9F7F9
:10285000E6E1F2E0DF011D928A95E9F780E090E081
:102860000E94451C873E9E4F21F40E94241C81112A
:1028700061C067EE7EEF80E090E00E94691C60E03E
:1028800082E090E00E944B1C60E083E090E00E94B8
:102890004B1C10922E0260E074E184E090E00E94F4
:1028A000691C60E086E090E00E944B1C6FEF87E0BF
:1028B00090E00E944B1C40E050E0BA0188E090E0BC
:1028C0000E945D1C60E08DE090E00E944B1C40E0A7
:1028D00050E0BA0188E190E00E945D1C60E087E171
:1028E00090E00E944B1C40E050E0BA018CE190E087
:1028F0000E945D1C60E070E080E290E00E94691C34
:1029000040E050E0BA0188E190E00E945D1C80E068
:102910000E94F51B0E94141C40E050E0BA018FE0B9
:1029200090E00E945D1C40E050E0BA0183E190E03D
:102930000E945D1C82E090E00E943D1C8093310269
:1029400084E090E00E94451C9093660180936501AD
:102950000E94B10EEFE1FEE43197F1F700C00000F4
:102960000E94B10E80914B0280FF08C06FEF7FEF95
:1029700080E090E00E94691C0E94A21983E090E030
:102980000E943D1C0E94C41781E091E09093930245
:10299000809392028E010F5F1F4FCE0149969CA734
:1029A0008BA780918C01853009F047C062E0F62E3C
:1029B00080918C01853009F03CC080918C0184307D
:1029C00021F110929602A8E1B0E0E0E40FB6F8948D
:1029D000A895A09360000FBEE093600083B7817F4D
:1029E000846083BF83B7816083BF7894889583B701
:1029F0008E7F83BF0FB6F894A895809160008861A0
:102A000080936000109260000FBE80918B0188233C
:102A100009F4CECF0E94B10EEBE4F2E081919191E6
:102A2000892B09F0D1C183E692E08E179F07B1F799
:102A3000BFCF0E94FE170E94D41A0E94B10E42E33B
:102A4000C42E42E0D42E5BE4E52E52E0F52E2AE4BB
:102A500032E0D701F601419151918D919D918427EA
:102A600095272E173F0719F0892BA9F322C0892B30
:102A700001F50E94F8196C0180912F0290913002AB
:102A8000C816D90609F457C08FEF89A38AA31BA2E1
:102A90000E94F8198160782F9DA38CA349A15AA1A7
:102AA0006BA18DA10E94E402D0923002C0922F024D
:102AB00042C03BE4432E32E0532E312CD2018D90A4
:102AC0009D902D01F6016080718068247924611445
:102AD000710441F1212CAA24A394B12CC3018A21B1
:102AE0009B21892BB1F02EA23FA221E0C4018A21B3
:102AF0009B21892B09F420E028A70E94F819816006
:102B0000782F9AA789A74EA15FA168A58AA50E94E0
:102B1000E4022394AA0CBB1CF9E02F12DFCFD601EC
:102B20008D929C923394B2E0CB0ED11CECE03E121D
:102B3000C5CF0E94EC190E94D41A90914A028917BD
:102B400021F080934A020E94EC1980918C0184301C
:102B500009F027CF83E08093E9008091E80082FFAD
:102B600020CF8091E80085FF23C00E94220E8111B2
:102B70001DC080E2C82ED12CCE0101965C0109C097
:102B80008091F100D5018D935D01B1E0CB1AD108A0
:102B900069F08091E80085FDF3CF8091E8008B77A4
:102BA0008093E8000E94220E882399F391E001C0EF
:102BB00090E08091E8008B778093E800992309F4F6
:102BC000F0CEE9818E2F90E0FC013197E331F105E1
:102BD00008F0F1C0EB56FF4F0C947F1C1A828BE07B
:102BE00055C08A81823009F405C150F4813009F062
:102BF000E2C00E94EC199B838C837D836E83DDC0D1
:102C0000833041F0843009F0D6C01B821C821D82C3
:102C10001E82D3C0FE013196D7018C9111969C91F2
:102C2000B2E0EB0EF11C9283838332968BA59CA5B8
:102C30008E179F0789F7C1C08A81823021F08530C5
:102C400009F4BBC0B8C06B817C818D819E810E94DC
:102C5000851C0E94F01BB1C04C816B818A810E944F
:102C6000C21B9D83CEC02D813E8132272327322770
:102C70004C816B818A810E94661B9FC00E948D1BC4
:102C80009CC080E152C082E08A838AE28B8395C037
:102C9000EA80FB80FE24EF24FE24AC80B12C680186
:102CA000C7018A529E4F9601201B310B2A153B0506
:102CB00008F083C0AAE2EA16A2E0FA0628F40E940D
:102CC0003D1CF601848303C0D60114961C92BFEF0D
:102CD000EB1AFB0AEFEFCE1ADE0AE2CFEA80FB80A6
:102CE000FE24EF24FE24AC80B12C6801C7018A5277
:102CF0009E4F9601201B310B2A153B0508F05DC045
:102D0000FAE2EF16F2E0FF0628F4D60114966C9171
:102D10000E944B1CBFEFEB1AFB0AEFEFCE1ADE0A44
:102D2000E5CF0E94561B49C082E08A8346C0EA80F4
:102D3000FB80FE24EF24FE24AC80B12C6801C70187
:102D400086969601201B310B2A153B05B0F5F0EB5A
:102D5000EF16F1E0FF0630F40E943D1CD6011496F8
:102D60008C9302C0F6011482FFEFEF1AFF0A2FEFD7
:102D7000C21AD20AE4CFEA80FB80FE24EF24FE24AC
:102D8000AC80B12C6801C70186969601201B310BDF
:102D90002A153B0590F4A0EBEA16A1E0FA0620F410
:102DA000F60164810E944B1CFFEFEF1AFF0A2FEF20
:102DB000C21AD20AE8CF8FEF898340E250E0B8010F
:102DC00082E00E946419EDCD19BCF9BC09B400FE83
:102DD000FDCF8091D8008F7D8093D8008091E00056
:102DE00082608093E0008091E00081FDFCCF0E9432
:102DF000FE17DECD85E290E00E943D1C1B821C8206
:102E00001D828E83DACFCF92DF92FF920F931F93B2
:102E1000CF93DF936C010091960180912E02082BD5
:102E2000C7E0D0E010E0C8010C2E02C09595879550
:102E30000A94E2F780FD04C02197A8F7F12C09C09D
:102E4000FC2EB6018C2F0E94710F0E947F0F0197FC
:102E500099F38F2DDF91CF911F910F91FF90DF900C
:102E6000CF900895CF93DF93EC010E940317BE012A
:102E70000E94710F0E947F0FDF91CF910895292F3B
:102E80009C3078F5893068F590E039E0239F800D1B
:102E9000911D1124682F677023E0969587952A95D8
:102EA000E1F7FC01EE0FFF1FE80FF91FED59FD4F91
:102EB00040E050E080E0219130E0062E02C03695DF
:102EC00027950A94E2F721703327042E01C0220FC0
:102ED0000A94EAF7822B4F5F5F4F4330510559F751
:102EE000089580E00895292F9C3088F5893078F581
:102EF00090E039E0239F800D911D1124282F277029
:102F000051E001C0550F2A95EAF723E09695879581
:102F10002A95E1F7FC01EE0FFF1FE80FF91FED59AD
:102F2000FD4F20E030E070E04081CB01022E02C076
:102F3000969587950A94E2F7817081958427852379
:102F4000842781932F5F3F4F2330310569F7089520
:102F500080939601089521E030E001C0220F8A9508
:102F6000EAF720958091960182230E94A817089580
:102F700021E030E001C0220F8A95EAF780919601A6
:102F8000822B0E94A817089580932E020895CF9354
:102F9000FC018081918123813481232B31F09F3F7B
:102FA00031F491E08F3F19F403C091E001C090E04B
:102FB000C92FC17090FD1CC0808191810E94321781
:102FC00092959F70963079F010F4925001C09A500B
:102FD000923088F4803F71F018F4883E60F40AC0A3
:102FE000843F49F407C0883E28F0813F21F402C0A5
:102FF000C0E001C0C1E08C2FCF9108951092110262
:1030000080910001882331F08091650187FF02C023
:103010008EE101C086E0E9E9F1E0DF011D928A95C9
:10302000E9F780E090E00E94AF1A80E090E00E9413
:103030008A1A109210020E942A110895882321F002
:103040000E9423110E942A110895882339F090913B
:103050001102892B809311020E942A11089588235E
:1030600009F455C0682F823869F40E94D41A81FF90
:103070004EC069E387E991E00E94551A0E942A1127
:1030800069E30EC0833899F40E94D41A80FF3FC0D0
:1030900063E587E991E00E94551A0E942A1163E5D1
:1030A00087E991E00E942D1A0E942A110895843820
:1030B00069F40E94D41A82FF2AC067E487E991E08C
:1030C0000E94551A0E942A1167E4EACF8CEF860FFE
:1030D000813A30F380E2860F883048F4677081E0EF
:1030E00001C0880F6A95EAF70E942311DDCF8BE5B6
:1030F000860F833028F480E090E00E94AF1A089594
:10310000685A693120F480E090E00E948A1A08959C
:10311000CF93882309F4B4C0C82F8238B1F40E9439
:10312000D41A81FDADC069E387E991E00E94551A88
:103130000E942A112FEF83EF91E0215080409040B0
:10314000E1F700C0000069E317C08338E1F40E9492
:10315000D41A80FD95C063E587E991E00E94551A75
:103160000E942A112FEF80E792E02150804090408A
:10317000E1F700C0000063E587E991E00E942D1AA5
:103180000E942A117DC08438B1F40E94D41A82FDB5
:1031900077C067E487E991E00E94551A0E942A11DE
:1031A0002FEF80E792E0215080409040E1F700C08F
:1031B000000067E4E1CF8CEF8C0F813AB8F5809185
:1031C00000018823E1F08091650187FF18C0EC2F92
:1031D000E695E695E695F0E0E956FE4F8281282FC8
:1031E00030E04C2F477081E090E002C0880F991FBB
:1031F0004A95E2F782239323892B59F411C0E9E918
:10320000F1E08191C81729F021E0EF39F207C9F701
:1032100007C06C2F87E991E00E942D1A0E942A11A5
:103220006C2F87E991E00E94551AAACF80E28C0F9B
:10323000883068F4C77081E090E001C0880FCA95BB
:10324000EAF790911102892B8093110299CFEBE557
:10325000EC0FE33040F4F0E0E85EFE4F808190E058
:103260000E94AF1A0DC0C85AC93150F4EC2FF0E0DB
:10327000EE0FFF1FE55EFE4F808191810E948A1A4A
:10328000CF9108951F93CF93DF93182F893319F0AF
:10329000C0E0D0E002C0C0E5D0E0812F0E948818D5
:1032A000209741F08FEC97E00197F1F700C0000004
:1032B0002197F6CF812F0E942F18DF91CF911F9178
:1032C00008958091690108950F931F93CF93DF9321
:1032D0008B01EA0190918C01943079F58F70809385
:1032E000E9008FEF9091E800815095FD06C09AE6C5
:1032F0009A95F1F700C08111F5CF8091E80085FF24
:103300001CC00E94220E882361F08091E8008E7715
:103310008093E80012C0F80181918F018093F10041
:103320002197209791F38091E80085FDF4CF80915B
:10333000E8008E778093E800E4CFDF91CF911F9172
:103340000F91089581E08093E00080E28093D8009F
:103350001092C9008FE097E20197F1F700C00000DA
:1033600087E090EBDC0180939B0290939C02A093FA
:103370009D02B0939E029CE088E10FB6F894A89558
:10338000809360000FBE90936000FFCF78941F92EF
:103390000F920FB60F9211248F939F93AF93BF9309
:1033A0008091970290919802A0919902B0919A020F
:1033B0000196A11DB11D8093970290939802A0934E
:1033C0009902B0939A02BF91AF919F918F910F9004
:1033D0000FBE0F901F9018952FB7F8946091970229
:1033E000709198028091990290919A022FBF08954E
:1033F0002FB7F8948091970290919802A09199022A
:10340000B0919A022FBF08951F920F920FB60F929C
:1034100011248F939F93AF93BF9380919602811154
:1034200013C08091970290919802A0919902B09157
:103430009A024196A11DB11D809397029093980224
:10344000A0939902B0939A02BF91AF919F918F91EF
:103450000F900FBE0F901F9018952091000122230E
:10346000C9F02091650127FF15C0262F26952695C6
:1034700026952E31C8F4FC01E20FF11D677081E042
:1034800090E001C0880F6A95EAF7809592818923C0
:1034900082830895FC0106962281621301C0128284
:1034A0003196E817F907C1F708952091000122230A
:1034B000C1F02091650127FF14C0262F269526957F
:1034C00026952E3130F5FC01E20FF11D677081E089
:1034D00090E001C0880F6A95EAF79281892B828378
:1034E0000895FC0132962FEF30E04191641789F086
:1034F0002F3F19F4411101C0232F3F5F3630A9F748
:103500002F3F39F0FC01E20FF11D27FDFA95628390
:1035100008950895A3E0B0E0E0E9FAE10C949C1C62
:10352000209194023091950228173907A1F09093C9
:10353000950280939402E0919202F0919302309769
:1035400051F024E029839B838A830680F781E02D54
:10355000CE01019609952396E2E00C94B81CA3E0F5
:10356000B0E0E5EBFAE10C949C1C209190023091C4
:10357000910228173907A1F090939102809390024D
:10358000E0919202F0919302309751F023E0298369
:103590009B838A830680F781E02DCE0101960995F1
:1035A0002396E2E00C94B81CE0919202F091930211
:1035B000309729F00190F081E02D0995089580E081
:1035C00008950F931F93CF93DF93C42F122FFC0105
:1035D00082818823B1F040938F020E94F819909362
:1035E0008E0280938D0280E28C0F883008F059C0E3
:1035F000C77081E001C0880FCA95EAF70E942518BC
:1036000050C080918F0248133CC020918D023091B0
:103610008E024FB7F8948091970290919802A091F2
:103620009902B0919A024FBF821B930B883C91057F
:1036300040F5D0E2D10FC117B9F080E28C0F88308D
:1036400040F4C77081E001C0880FCA95EAF70E9474
:103650001E18D83018F581E0912F977001C0880F9F
:103660009A95EAF70E942518802F0E944219D830B7
:10367000C0F4212F277081E001C0880F2A95EAF756
:103680000AC080E28C0F883060F4C77081E001C00E
:10369000880FCA95EAF70E941E1803C0802F0E9467
:1036A0004219DF91CF911F910F910895CF93DF932E
:1036B000C6EDD1E060E0CE010E944B1C2196C11501
:1036C00084E0D807B9F7DF91CF9108951F93CF9386
:1036D000DF93962F8230E8F46C30D8F44930C8F488
:1036E000632F122FC42FD0E0CC0FDD1F22E1929F59
:1036F000C00DD11D112498ED899FC00DD11D11243D
:10370000CE0186960E944B1C612FCE0187960E94A7
:103710004B1CDF91CF911F910895A0E0B0E0E3E949
:10372000FBE10C94941CA12CE12CF12CB12C00E0B9
:1037300010E0C0E0D0E06701C00ED11EFE01EE0F28
:10374000FF1FEC0DFD1DE858FC4F259134914C2FC7
:103750006B2D8A2D0E94661B2196C930D10571F709
:103760000E5E1F4FB3948CE0B812E3CF88EDE80EE5
:10377000F11CA39482E0A812D9CFCDB7DEB7EAE05E
:103780000C94B01C0F931F93CF93DF93823008F5F6
:103790006C30F8F44930E8F4C42FD0E0CC0FDD1FD2
:1037A00022E1629FC00DD11D112438ED839FC00D11
:1037B000D11D1124CE0186960E943D1C90E0182F49
:1037C0000027CE0187960E943D1C9801282BC90135
:1037D00002C080E090E0DF91CF911F910F9108959A
:1037E00085E290E00E944B1C0895CF93C82F811171
:1037F00002C06FEF01C062E282E290E00E944B1CC7
:10380000C11102C06FEF01C062E183E290E00E944B
:103810004B1CC11102C06FEF01C068E084E290E070
:103820000E944B1CCF91089580E00E94F51B60E040
:1038300070E0CB010E94F01B0E948D1B0E94561B62
:1038400081E00E94F51B089582E290E00E943D1CF9
:10385000823281F483E290E00E943D1C823151F477
:1038600084E290E00E943D1C91E0883009F090E0F5
:10387000892F01C080E081700895F999FECF92BD33
:1038800081BDF89A992780B50895A8E1B0E042E09B
:1038900050E00C94711C262FF999FECF92BD81BD8A
:1038A000F89A019700B4021639F01FBA20BD0FB67E
:1038B000F894FA9AF99A0FBE08950396272F0E945A
:1038C0004C1C0E944B1C252F0E944C1C242F0C9436
:1038D0004C1C0196272F0E944C1C0C944B1CDC01A5
:1038E000CB01FC01F999FECF06C0F2BDE1BDF89A0B
:1038F000319600B40D9241505040B8F70895EE0F44
:10390000FF1F0590F491E02D0994692796276927F8
:1039100078278727782708952F923F924F925F92BA
:103920006F927F928F929F92AF92BF92CF92DF92CF
:10393000EF92FF920F931F93CF93DF93CDB7DEB734
:10394000CA1BDB0B0FB6F894DEBF0FBECDBF0994C8
:103950002A88398848885F846E847D848C849B841F
:10396000AA84B984C884DF80EE80FD800C811B812D
:10397000AA81B981CE0FD11D0FB6F894DEBF0FBE5C
:10398000CDBFED010895FB01DC0104C08D910190D4
:10399000801921F441505040C8F7881B990B0895B5
:0439A000F894FFCFC9
:1039A40001611995098D098E0940226D8F026D02FE
:1039B4000002E102FA021A03818283E200E900EACA
:1039C40000B500B600B700CD008301CC008A019297
:1039D4000194012102230224022502260227022A3D
:1039E40002B300B4006F0070009F01CB0192919369
:1039F400909530F0F1F7F467669697343536F6F51E
:023A0400C69466
:00000001FF
